:020000040000FA
:100000000CEF00F0FFFFFFFFD8CFFFF5E0CF0DF0C2
:10001000D5EF01F0FFFFFFFF00EE0EF010EE0FF046
:1000200069EC23F000EEAAF011EE00F069EC23F089
:1000300005EE25F015EEFDF069EC23F015EF06F066
:10004000FFFF33D093688B8800F000F00EA001D042
:1000500001D019D08B8A00F000F000F000F0815040
:100060000001E36F8B9AE339F00BF00BE26F8B8AA0
:1000700000F000F000F000F08150E36F8B9AE35144
:100080000F0BE2130BD08B8A00F000F000F000F0B1
:1000900081500001E36F8B9AE351E26F8B98936A72
:1000A0000001E25100D01200FFFFCCD7FFFF1ED0AD
:1000B0000001E80EDF6F030EE06F07D0C1DFE16FD4
:1000C000E1BF01D001D001D00FD00001DF51006E9F
:1000D000E051016E010EDF5F000EE05B0150001089
:1000E000D8A401D001D0EAD71200FFFFE1D7FFFF6B
:1000F00027D00001D36FDADF0EA001D001D015D0D8
:100100000001D3390F0B0F0B8A6E8B8A00F000F0C1
:1001100000F000F08B9AD3510F0B8A6E8B8A00F09F
:1001200000F000F000F08B9A09D00001D3518A6EE4
:100130008B8A00F000F000F000F08B9A1200FFFFB5
:10014000D8D7FFFF2CD00001DE6FB0DF8A6A8B8624
:100150000EA001D001D017D00001DE390F0B0F0B1C
:100160008A128B8A00F000F000F000F08B9AF00EFB
:100170008A16DE510F0B8A128B8A00F000F000F015
:1001800000F08B9A09D00001DE518A6E8B8A00F054
:1001900000F000F000F08B9A8B961200FFFFD3D78F
:1001A000DC00FFFF2ED016D00001DCC0F6FFDDC062
:1001B000F7FF010EDC27000EDD23050EF76404D0E7
:1001C0000800FFFFF55005D0F6CFE9FFF7CFEAFFB3
:1001D000EF50B7DFDCC0F6FFDDC0F7FF050EF764B8
:1001E00004D00800FFFFF55005D0F6CFE9FFF7CFA8
:1001F000EAFFEF500009D8A401D001D0D5D71200F2
:10020000FFFFD1D7FFFF5AD00E900001D16FD1511F
:10021000D8A401D001D004D00E80030ED06F03D03B
:10022000380E0001D06F8B968B9A8B989496949A87
:1002300094988A6A936A140E96EC02F00001D051E9
:100240008A6E8B8A00F000F000F000F08B9A050EA9
:1002500096EC02F00001D0518A6E8B8A00F000F01B
:1002600000F000F08B9A140EBAEC02F00001D051AD
:100270008A6E8B8A00F000F000F000F08B9A050E79
:10028000BAEC02F00EA001D001D00CD00FDF020EAC
:100290008A6E8B8A00F000F000F000F08B9A280E36
:1002A00026DF02D0380E23DF0F0E21DF010E1FDF05
:1002B000060E1DDF800E1BDF1200FFFFA5D7FFFF1C
:1002C00073D0F2AA05D000D0F2A402D000D002D0A0
:1002D00000D060D0F2948B903C0E921280CF00F050
:1002E000D8900032D8900030FF0A0F0B0001FF6F4A
:1002F0000501F953D8B401D001D006D00501010E93
:10030000F95F0501F76B02D0FFC0F7F50001FF515F
:10031000D8A401D001D005D00501F96B0501F86B17
:1003200009D0FA0E0501F86101D001D003D0050112
:10033000010EF8270501F553D8B401D001D003D040
:100340000501010EF55F0501FC53D8B401D001D0C1
:1003500003D00501010EFC5F0501F453D8B401D0B0
:1003600001D004D00501010EF45F01D08990F30E95
:10037000D76ECB0ED66E0501FB53D8A401D001D0A9
:1003800006D0F6C5FBF5010EE8CFFAF503D005015E
:10039000010EFB5FFDC500F0FEC5E8FF0DC0E0FFEC
:1003A000FFC5D8FF1000FFFF8CD7FFFFE8CFFEF599
:1003B00000C0FDF584D7FFFF15D0F168050ED56E9E
:1003C000F30ED76ECB0ED66E080EE8CFF6F5F6C557
:1003D000FBF50501FA6B0501F96B0501F56BF28A76
:1003E0001200FFFFEAD7FFFFE96AEA6AFFFF0C6A23
:1003F000FFFF086A096A0A6A0B6A045005100610B2
:10040000071006E1046A056A066A076A2BEF23F003
:10041000C00E0C1606D0D8900436053606360736C0
:100420000C2A07AEF8D70C2AD890083609360A36B7
:100430000B360750035C08E10650025C05E10550ED
:10044000015C02E10450005C09E308800450005E96
:100450000550015A0650025A0750035AD8900732E5
:100460000632053204320C060C503F0BDDE10CBCA9
:100470005DEC23F00050046E0150056E0250066ED4
:100480000350076E0850006E0950016E0A50026E4C
:100490000B50036E0CAE30EF23F05DEC23F030EF29
:1004A00023F0FFFFE96AEA6AFFFF0050086E01507F
:1004B000096E02500A6E03500B6E026A036A0850FE
:1004C0000402F3CF00F0F4CF01F00502F35001264F
:1004D000F450022209500402F3500126F450022283
:1004E000D8B0032A08500602F3500226F450032223
:1004F00009500502F3500226F45003220A50040268
:10050000F3500226F450032208500702F35003264A
:1005100009500602F35003260A500502F350032641
:100520000B500402F350032630EF23F0FFFF21D0DD
:100530000001D46F15D00001F80ED26F010ED36FF9
:1005400000D00001D251006ED351016E010ED25F76
:10055000000ED35B01500010D8A401D001D0F1D718
:100560000001D407D429D8A401D001D0E4D71200C7
:10057000FFFFDED7FFFF17D00001D36F0BD0080EAF
:100580000001D26F00D00001D207D229D8A401D037
:1005900001D0F9D70001D307D329D8A401D001D0C5
:1005A000EED71200FFFFE8D7DE00FFFFDEC0D9FF65
:1005B000DFC0DAFF0001E0C0F6FFE1C0F7FFE02B8B
:1005C000000EE123D9CFE9FFDACFEAFFD94ADA2AD0
:1005D000050EF76403D00800F55005D0F6CFE1FF13
:1005E000F7CFE2FFE750EF6EEF50D8A4E3D7DEC0BD
:1005F00000F0DFC001F01200FFFFD8D7FFFFFFFFC0
:1006000072706D006D5620004B6720002520200081
:10061000434120002D424400755320006D532000BB
:100620004B6D200020202000032020006D48670033
:100630006D560000252020002020200020202000D2
:1006400020202000562020006C706D0000004553D3
:1006500050454400070001024D4146530000070386
:100660000204544852000000070303065754454D46
:1006700050000B0A04084954454D50000B0A050A66
:10068000495052455300070B060C4146000000003C
:100690000709070E4554454D5000070A08104650FB
:1006A00052455300070209125642415454000911A1
:1006B0000A1456535045440007080B1653570000C0
:1006C000000003090C1844455350440000030D1A60
:1006D00044544852000000030E1C4B4E4F434B0045
:1006E00007090F204655454C31000706102249479F
:1006F0004E503100000511244655454C3200070686
:10070000122649474E5032000005132849534356DC
:1007100000000103142A5457494E0000010315320A
:100720004643544F54000109163446434D4150008E
:100730000109173646435448520001091838464308
:10074000565350000109193A4643575450000109C5
:100750001A3C46434954500001091B3E4643455448
:10076000500001091C4046434650520001091D42F9
:100770004643564F4C0001091E4446434C4F44002B
:1007800001091F46464341434300010920484643AF
:10079000444543000109214A46435354410001099D
:1007A000224C464341494A000109234E4643494EE3
:1007B0004A0001092450464349444C00010925627E
:1007C00049524D4150000A0926634952544852008B
:1007D0000A0927644952565350000A0928654952AC
:1007E000575450000A0929664952495450000A09D1
:1007F0002A674952455450000A092B68495246500D
:1008000052000A092C694952564F4C000A092D6AB8
:1008100049524C4F44000A092E6B49524143430050
:100820000A092F6C4952444543000A09306D495268
:10083000535441000A09316E495249444C000A0997
:10084000326F4947444953000A0933784F324143D4
:100850005400030934794143535700000309357AA2
:100860004C44535731000309367B4C4453573200F4
:100870000309377C4E54524C0000030900204553B5
:1008800050454400070001224950524553000402DC
:1008900002245448520000000103032644544852E5
:1008A0000000010304284D41465331000701052A89
:1008B0004D41465332000701062E56535045440021
:1008C000070807304146000000000509083246319C
:1008D000494E0000000609344632494E0000000926
:1008E0000A3846314F55540000060B3A46324F55F0
:1008F000540000060C3E4149434F000000060D42E3
:1009000041494344000000060E44564241545400FD
:1009100005110F46564F5054310000011048564FF4
:10092000505432000006114A5754454D50000B0AEE
:10093000124C4954454D50000B0A134E46544F5427
:1009400000000209144F49544F5400000609155085
:1009500041544F5400000209165146434F52310092
:100960000209175246434F523200020918534643B8
:100970005754500002091954464349545000020983
:100980001A5546434743430002091B5646435650F7
:10099000430002091C5746435342430002091D58B5
:1009A00046434143430002091E59495231000000A9
:1009B00006091F5A4952320000000609205B4952BD
:1009C000575450000609215C495249545000060909
:1009D000225D4952474343000609235E495256505F
:1009E00043000609245F495253424300060925602B
:1009F000495241434300060926614157544D500076
:100A0000020927624149544D50000209286354539A
:100A1000424300000209005045535045440007007E
:100A200001524D41465300000712025454485200EF
:100A30000000070303565754454D5000080A045858
:100A40004954454D50000801055A4950524553003C
:100A50000402065C4146000000000509075E45549B
:100A6000454D5000000A08704454485200000003ED
:100A7000097256424154540009110A7A565350459E
:100A8000440007080B604655454C310007060C62D0
:100A900049474E50310000050D764655454C320011
:100AA00007060E7849474E50320000050F7E495325
:100AB000435620000709106C4552523100000709C7
:100AC000116E4552523200000709004014540A4A80
:100AD0001E5E18180E1010110E00181418151705A8
:100AE00005005650524F332E3178005650524F3336
:100AF0002E3078005650524F322E78002020496E0A
:100B000074657276616C002046434F4E2074797094
:100B100065005761726E4C454420736574204D6FBB
:100B2000646500202038204D6F6E69746F72204D0F
:100B30006F646500203220426172477261706820E4
:100B40004D6F6465002034205065616B486F6C64A4
:100B5000204D6F64650020202053455455502020BF
:100B600020204D6F646500202534646D530046439A
:100B70004F4E2D53005345545550004D4F44452082
:100B800050434C5220202055502020444F574E00B7
:100B90004D4F4445202053454C20202055502020C7
:100BA000444F574E0046434F4E204D6F6E69746F51
:100BB0007220566572312E3000416C6C205269678C
:100BC0006874732052657365727665642E00202008
:100BD000202D2D2D0020202020203230303328637E
:100BE00029204B617368692E2C0042617220536387
:100BF000616C652000202D2D2D20002534750025E9
:100C0000346400253364002532642E2530326400BC
:100C1000256325642E25303264002532642E25316B
:100C200064004F4E004F46460000FFFF64EF16F091
:100C3000A66AAC6AAB6AC66A96928D8294908B90D3
:100C400096948D9489908992929092929284010EBA
:100C500002EC01F04AEC1BF0DBEC01F00C0E77EC3F
:100C600000F0020E77EC00F00001A50EDC6F0B0E19
:100C7000DD6FD1EC00F0940E77EC00F00001D50EA2
:100C8000DC6F0B0EDD6FD1EC00F0D40E77EC00F0D2
:100C90000001B90EDC6F0B0EDD6FD1EC00F000012E
:100CA000C06B1D0EC06501D001D001D00BD0640E09
:100CB00096EC02F0010E0001C0271D0EC06501D0A8
:100CC00001D0F5D7010E77EC00F00001C06B070EE4
:100CD000C06501D001D001D040D00001C051480F03
:100CE00077EC00F01B0EA1EC00F00001C051500F9A
:100CF00077EC00F0180EA1EC00F00001C051580F85
:100D000077EC00F0C0C000F0016A0050D20FF66E20
:100D10000150F76E0A0EF7220800FFFFF550A1EC14
:100D200000F00001C051600F77EC00F0C0C000F08F
:100D3000016A0050DA0FF66E0150F76E0A0EF722C4
:100D40000800FFFFF550A1EC00F0010E0001C027E4
:100D5000070EC06501D001D0C0D7080E0001D06FCA
:100D6000D16BFBEC22F0E8CFF6F50501FC0EF6178F
:100D7000040E0501F66101D005D0C80E0501F66527
:100D800002D000D002D000D00BD0080EE8CFF6F58C
:100D9000080E0001D06FD16B080ED26FBCEC1FF0B3
:100DA000090E0001D06FD16BFBEC22F0E8CF43F5C8
:100DB0001ED0360E0001C56F25D0270E0001C56F6D
:100DC00021D0360E0001C56F1DD0100E0001C56F79
:100DD00019D00501436B090E0001D06FD16BD26BA6
:100DE000BCEC1FF0360E0001C56F0CD00BD043C514
:100DF000E8FF000ADEE0010AE0E0030AE2E0010A9F
:100E0000E4E0E7D70001C06B070EC06501D001D058
:100E100001D029D00001C051D06FD16BFBEC22F082
:100E2000006E00C002F0036AC5C000F0016A015004
:100E3000800A046E0350800A045C02E10250005CE8
:100E4000D8B001D001D007D00001C051D06FD16B14
:100E5000D26BBCEC1FF0010E0001C027070EC0656D
:100E600001D001D0D7D70001C06B010EC06501D001
:100E700001D001D055D00001D890C035006E016A74
:100E800001360A0E0024D06F000E0120D16FFBEC5A
:100E900022F0006E0001C051020DAC0EF324E96E89
:100EA000000EF420EA6E00C0EFFFD890C035006E4F
:100EB000016A01360B0E0024D06F000E0120D16FA5
:100EC000FBEC22F0006E0001C051020DAD0EF324C8
:100ED000E96E000EF420EA6E00C0EFFFC051020D73
:100EE000AC0EF324E96E000EF420EA6EEE50ED1025
:100EF000D8A401D001D00CD0C051020DAC0EF32407
:100F0000E96E000EF420EA6E010EEE6E000EED6E3C
:100F1000010E0001C027010EC06501D001D0ABD782
:100F20000001C06B030EC06501D001D001D03AD0E2
:100F30000001D890C035006E016A0136120E0024FF
:100F4000D06F000E0120D16FFBEC22F0006E00018B
:100F5000C051020DB80EF324E96E000EF420EA6EC3
:100F600000C0EFFFD890C035006E016A0136130E45
:100F70000024D06F000E0120D16FFBEC22F0006E38
:100F80000001C051020DB90EF324E96E000EF420E9
:100F9000EA6E00C0EFFF010EC027030EC06501D04E
:100FA00001D0C6D71A0E0001D06FD16BFBEC22F036
:100FB0000001C36F040EC36501D001D001D0C36B23
:100FC000F28ED58E0001C06B010EC66F60EF16F079
:100FD0000001C351D8A401D001D03DD20C0E77EC52
:100FE00000F0010E77EC00F0C00E77EC00F000018D
:100FF000230EDC6F0B0EDD6FD1EC00F0D40E77EC1E
:1010000000F00001900EDC6F0B0EDD6FD1EC00F0F4
:101010003C0EE8CFFCF5010E0001C66FC26B899251
:1010200017D20001C651D8B407D000D00501FC5337
:10103000D8A402D000D002D000D063D0010E77EC4B
:1010400000F00001C06B070EC06501D001D001D0D7
:1010500045D00001C051D06FD16BFBEC22F0006E87
:101060000001C05105EE25F0E926000EEA2200C07D
:10107000EFFFC05105EE25F0E926000EEA22EF5001
:10108000C56101D001D00ED0C05105EE25F0E92692
:10109000000EEA22000EEF6EC051D06FD16BD26B02
:1010A000BCEC1FF0C0C000F0016A0050CA0FF66E21
:1010B0000150F76E0A0EF7220800FFFFF550800975
:1010C00077EC00F00001C05166EC16F0010E000153
:1010D000C027070EC06501D001D0BBD7C2C000F049
:1010E000016A0050CA0FF66E0150F76E0A0EF72221
:1010F0000800FFFFF550800977EC00F00001C66B97
:10110000C6D00501F7A501D001D045D00001C251DC
:1011100005EE25F0E926000EEA22EF50D8B401D002
:1011200001D007D0C25105EE25F0E926000EEA22D3
:10113000EF060501F76B140E0501F86501D001D02B
:1011400004D0080EE8CFF9F503D0140EE8CFF9F576
:101150000001C25166EC16F00001C251D06FD16B94
:10116000C25105EE25F0E926000EEA22EF50D26FBB
:10117000BCEC1FF0C2C000F0016A0050CA0FF66E4E
:101180000150F76E0A0EF7220800FFFFF5508009A4
:1011900077EC00F07CD00501F7A701D001D048D052
:1011A0000001C25105EE25F0E926000EEA22EF50BB
:1011B000006EC551005CD8B001D001D007D0C2513B
:1011C00005EE25F0E926000EEA22EF2A0501F76B6D
:1011D000140E0501F86501D001D004D0080EE8CF47
:1011E000F9F503D0140EE8CFF9F50001C25166EC11
:1011F00016F00001C251D06FD16BC25105EE25F03F
:10120000E926000EEA22EF50D26FBCEC1FF0C2C0FC
:1012100000F0016A0050CA0FF66E0150F76E0A0E18
:10122000F7220800FFFFF550800977EC00F02FD07F
:101230000501F7A301D001D02AD0070E0001C26139
:1012400001D001D003D0010EC22702D00001C26B31
:101250000501F76B140E0501F86501D001D004D02B
:10126000080EE8CFF9F503D0140EE8CFF9F5C2C0A7
:1012700000F0016A0050CA0FF66E0150F76E0A0EB8
:10128000F7220800FFFFF550800977EC00F0050118
:10129000F7A101D001D011D0010E0001C327140E17
:1012A000E8CFF9F50501F76B1A0E0001D06FD16B8D
:1012B000C351D26FBCEC1FF0CCD00001C651D8A4F2
:1012C00007D000D00501FA53D8B402D000D001D025
:1012D00006D00501F853D8A402D000D002D000D027
:1012E000B7D0080E98EC1AF00C0E77EC00F0050160
:1012F0004253D8B401D001D02AD00501426B00017D
:10130000C16B070EC16501D001D001D01FD0C1C093
:1013100000F0016A0050CA0FF66E0150F76E0A0E17
:10132000F7220800FFFFF550850F77EC00F0000171
:10133000F50EDC6F0B0EDD6FD1EC00F0010E00013D
:10134000C127070EC16501D001D0E1D76CD00001E3
:10135000C06BC16B070EC16501D001D001D05AD05E
:10136000C1C000F0016A0050CA0FF66E0150F76E5E
:101370000A0EF7220800FFFFF550850F77EC00F00A
:101380000001CA0EDC6F000EDD6FC70EDE6F000EAF
:10139000DF6FC15105EE25F0E926000EEA22EF507D
:1013A000F4EC16F0CAC0D7F0CBC0D8F00001C7519A
:1013B000D96F050EDA6FB1EC17F0040E0001C161B0
:1013C00001D001D01FD0CAC0DCF0CBC0DDF0C751C6
:1013D000FEEC19F00001C151020DB80EF324E96EC4
:1013E000000EF420EA6EEECF02F0EDCF03F00350D2
:1013F000015C02E10250005CD8A001D001D002D013
:10140000010EC06F010E0001C127070EC16501D09A
:1014100001D0A6D70001C051D8B401D001D002D06C
:10142000898201D089920501FA6BC2C000F0016A7D
:101430000050CA0FF66E0150F76E0A0EF722080030
:10144000FFFFF550800977EC00F00F0E77EC00F00D
:10145000E8D560EF16F00001C305D8A401D001D093
:10146000D1D20C0E77EC00F0010E77EC00F0C00E3C
:1014700077EC00F00001450EDC6F0B0EDD6FD1EC58
:1014800000F0D40E77EC00F000017B0EDC6F0B0E49
:10149000DD6FD1EC00F03C0EE8CFFCF5010E000151
:1014A000C66FC26B8992ABD20001C651D8B407D0C7
:1014B00000D00501FC53D8A402D000D002D000D047
:1014C00086D0010E77EC00F00001C06B030EC06502
:1014D00001D001D001D045D00001C051D06FD16BF7
:1014E000FBEC22F0006E0001C05105EE25F0E9266C
:1014F000000EEA2200C0EFFFC05105EE25F0E926FC
:10150000000EEA22EF50C56101D001D00ED0C051CB
:1015100005EE25F0E926000EEA22000EEF6EC0511E
:10152000D06FD16BD26BBCEC1FF0C0C000F0016A71
:101530000050CA0FF66E0150F76E0A0EF72208002F
:10154000FFFFF550800977EC00F00001C05166EC18
:1015500016F0010E0001C027030EC06501D001D0B6
:10156000BBD7C2C000F0016A0050CA0FF66E01502E
:10157000F76E0A0EF722040EF626000EF722080078
:10158000FFFFF550840F77EC00F00001C06B030EF5
:10159000C06501D001D001D014D00001C051020DAE
:1015A000B00EF324E96E000EF420EA6E000EEE6E2B
:1015B000000EED6E010EC027030EC06501D001D0F4
:1015C000ECD7010EE8CFFAF50001C66B11D1050189
:1015D000F7A501D001D059D00001C25105EE25F088
:1015E000E926000EEA22EF50D8B401D001D007D08E
:1015F000C25105EE25F0E926000EEA22EF060501AC
:10160000F76B140E0501F86501D001D004D0080E67
:10161000E8CFF9F503D0140EE8CFF9F5C2C000F019
:10162000016A0050CA0FF66E0150F76E0A0EF722DB
:101630000800FFFFF550800977EC00F00001C2516F
:1016400066EC16F00001C251D06FD16BC25105EEAD
:1016500025F0E926000EEA22EF50D26FBCEC1FF015
:10166000C2C000F0016A0050CA0FF66E0150F76E5A
:101670000A0EF722040EF626000EF7220800FFFFDE
:10168000F550840F77EC00F0B3D00501F7A701D037
:1016900001D05CD00001C25105EE25F0E926000E14
:1016A000EA22EF50006EC551005CD8B001D001D0E5
:1016B00007D0C25105EE25F0E926000EEA22EF2AF6
:1016C0000501F76B140E0501F86501D001D004D0B7
:1016D000080EE8CFF9F503D0140EE8CFF9F5C2C033
:1016E00000F0016A0050CA0FF66E0150F76E0A0E44
:1016F000F7220800FFFFF550800977EC00F00001A9
:10170000C25166EC16F00001C251D06FD16BC251CC
:1017100005EE25F0E926000EEA22EF50D26FBCEC70
:101720001FF0C2C000F0016A0050CA0FF66E0150EF
:10173000F76E0A0EF722040EF626000EF7220800B6
:10174000FFFFF550840F77EC00F052D00501F7A3AE
:1017500001D001D04DD0030E0001C26101D001D0F3
:1017600003D0010EC22702D00001C26B0001C06B82
:10177000030EC06501D001D001D014D00001C051CA
:10178000020DB00EF324E96E000EF420EA6E000E96
:10179000EE6E000EED6E010EC027030EC06501D087
:1017A00001D0ECD7010EE8CFFAF50501F76B140E66
:1017B0000501F86501D001D004D0080EE8CFF9F595
:1017C00003D0140EE8CFF9F5C2C000F0016A005052
:1017D000CA0FF66E0150F76E0A0EF722040EF626B7
:1017E000000EF7220800FFFFF550840F77EC00F0A1
:1017F0000501F7A101D001D011D0010E0001C327CE
:10180000080EE8CFF9F50501F76B1A0E0001D06F4D
:10181000D16BC351D26FBCEC1FF0F2D00001C651A6
:10182000D8A407D000D00501FA53D8B402D000D014
:1018300001D006D00501F853D8A402D000D002D0C0
:1018400000D0DDD0040E98EC1AF00C0E77EC00F00E
:1018500005014253D8B401D001D02AD00501426B12
:101860000001C16B030EC16501D001D001D01FD0B2
:10187000C1C000F0016A0050CA0FF66E0150F76E49
:101880000A0EF7220800FFFFF550850F77EC00F0F5
:101890000001CE0EDC6F0B0EDD6FD1EC00F0010EFF
:1018A0000001C127030EC16501D001D0E1D78ED060
:1018B0000001C06BC16B030EC16501D001D001D026
:1018C0007CD0C1C000F0016A0050CA0FF66E015012
:1018D000F76E0A0EF7220800FFFFF550850F77EC30
:1018E00000F00001CA0EDC6F000EDD6FC70EDE6F68
:1018F000000EDF6FC15105EE25F0E926000EEA2249
:10190000EF50F4EC16F0CAC0D7F0CBC0D8F000010D
:10191000C751D96F060EDA6FB1EC17F00001C15153
:1019200005EE25F0E926000EEA22EF5066EC19F0EC
:10193000C1C000F0016A0050CA0FF66E0150F76E88
:101940000A0EF722040EF626000EF7220800FFFF0B
:10195000F550840F77EC00F00001C15106EC19F04E
:10196000040E0001C16101D001D01FD0CAC0DCF05B
:10197000CBC0DDF0C751FEEC19F00001C151020DE2
:10198000B80EF324E96E000EF420EA6EEECF02F0FA
:10199000EDCF03F00350015C02E10250005CD8A0DF
:1019A00001D001D002D0010EC06F010E0001C1278D
:1019B000030EC16501D001D084D70001C051D8B455
:1019C00001D001D002D0898201D089920501FA6B41
:1019D000C2C000F0016A0050CA0FF66E0150F76EE7
:1019E0000A0EF722040EF626000EF7220800FFFF6B
:1019F000F550840F77EC00F00F0E77EC00F054D523
:101A000060EF16F00001C351020AD8A401D002D041
:101A10004FEF11F00C0E77EC00F0010E77EC00F0B8
:101A2000C00E77EC00F00001340EDC6F0B0EDD6FA2
:101A3000D1EC00F0D40E77EC00F00001900EDC6FDA
:101A40000B0EDD6FD1EC00F03C0EE8CFFCF5010E83
:101A50000001C66FC26B89924BEF11F00001C651B5
:101A6000D8B407D000D00501FC53D8A402D000D0D0
:101A700002D000D070D0010E77EC00F00001C06BF6
:101A8000010EC06501D001D001D048D00001C05185
:101A9000D06FD16BFBEC22F0006E0001C05105EE5F
:101AA00025F0E926000EEA2200C0EFFFC05105EE46
:101AB00025F0E926000EEA22EF50C56101D001D0E1
:101AC0000ED0C05105EE25F0E926000EEA22000EE8
:101AD000EF6EC051D06FD16BD26BBCEC1FF0000128
:101AE000D890C035006E016A01360050CA0FF66EFC
:101AF0000150F76E0A0EF7220800FFFFF55080092B
:101B000077EC00F00001C05166EC16F0010E000108
:101B1000C027010EC06501D001D0B8D70001D89010
:101B2000C235006E016A01360050CA0FF66E0150D0
:101B3000F76E0A0EF722040EF626000EF7220800B2
:101B4000FFFFF550890F77EC00F0010EE8CFFAF5B2
:101B50000001C66B8DD20501F7A501D001D004D1DB
:101B60000001CA0EDC6F000EDD6FC70EDE6F000EC7
:101B7000DF6FC25105EE25F0E926000EEA22EF5094
:101B8000F4EC16F00001C7512DEC1AF000C0C8F0BB
:101B900001C0C9F00001C251020DAC0EF324E96E80
:101BA000000EF420EA6EEECF00F0EDCF01F0C95147
:101BB000015C02E1C851005CD8B001D001D00CD06A
:101BC000000EC95D020ED8B4C85DD8A001D001D006
:101BD00003D0D890C933C8330001C251020DAC0EF6
:101BE000F324E96E000EF420EA6EEECF00F0EDCFA4
:101BF00001F00150C95D02E10050C85DD8B001D0CC
:101C000001D00CD0C251020DAC0EF324E96E000ECF
:101C1000F420EA6EC851EE5EC951ED5A0501F76B2A
:101C2000140E0501F86501D005D0780E0501F861A4
:101C300002D000D002D000D004D0040EE8CFF9F5D5
:101C40000DD0780E0501F86501D001D004D00A0E40
:101C5000E8CFF9F503D0140EE8CFF9F5010E000135
:101C6000C66F140EE8CFFCF5D890C235006E016A3D
:101C700001360050CA0FF66E0150F76E0A0EF722B9
:101C80000800FFFFF550800F77EC00F00001EA0E2E
:101C9000DC6F0B0EDD6FD1EC00F00001C251020DC4
:101CA000AC0EF324E96E000EF420EA6EEECFD0F015
:101CB000EDCFD1F0C751C6EC19F000C0CCF001C097
:101CC000CDF0CCC0D7F0CDC0D8F00001C751D96F4E
:101CD000060EDA6FB1EC17F00001D890C235006E35
:101CE000016A01360A0E0024D06F000E0120D16F68
:101CF000C251020DAC0EF324E96E000EF420EA6E20
:101D0000EF50D26FBCEC1FF00001D890C235006ECE
:101D1000016A01360B0E0024D06F000E0120D16F36
:101D2000C251020DAD0EF324E96E000EF420EA6EEE
:101D3000EF50D26FBCEC1FF00001D890C235006E9E
:101D4000016A01360050CA0FF66E0150F76E0A0E96
:101D5000F722040EF626000EF7220800FFFFF550CA
:101D6000890F77EC00F084D10501F7A701D001D0ED
:101D700049D10001CA0EDC6F000EDD6FC70EDE6FA9
:101D8000000EDF6FC25105EE25F0E926000EEA22B3
:101D9000EF50F4EC16F00001C7512DEC1AF000C022
:101DA000C8F001C0C9F00001C251020DAC0EF3240D
:101DB000E96E000EF420EA6EEECF02F0EDCF03F0F4
:101DC000FF0E006EFF0E016EC851005EC951015A30
:101DD0000350015C02E10250005CD8B001D001D098
:101DE0000CD0000EC95D020ED8B4C85DD8A001D0D9
:101DF00001D003D0D890C933C833FF0E006EFF0E58
:101E0000016E0001C851005EC951015AC251020D54
:101E1000AC0EF324E96E000EF420EA6EEECF02F071
:101E2000EDCF03F00150035C02E10050025CD8B03A
:101E300001D001D00CD0C251020DAC0EF324E96EDA
:101E4000000EF420EA6EC851EE26C951ED220501BC
:101E5000F76B140E0501F86501D005D0780E050169
:101E6000F86102D000D002D000D004D0040EE8CF38
:101E7000F9F50DD0780E0501F86501D001D004D038
:101E80000A0EE8CFF9F503D0140EE8CFF9F5010EEC
:101E90000001C66F140EE8CFFCF5D890C235006E75
:101EA000016A01360050CA0FF66E0150F76E0A0E35
:101EB000F7220800FFFFF550800F77EC00F00001DB
:101EC000EA0EDC6F0B0EDD6FD1EC00F00001C751A4
:101ED000020AD8A401D005D0C751060AD8A402D05E
:101EE00000D007D000D00001C7510A0AD8A402D000
:101EF00000D002D000D01FD00001C251020DAC0EA4
:101F0000F324E96E000EF420EA6EEE52010EED5C51
:101F1000000ED8B4EF5CD8A001D001D00CD0C251D3
:101F2000020DAC0EF324E96E000EF420EA6EFF0EF3
:101F3000EE6E000EED6E0001C251020DAC0EF324E8
:101F4000E96E000EF420EA6EEECFD0F0EDCFD1F0C6
:101F5000C751C6EC19F000C0CCF001C0CDF0CCC028
:101F6000D7F0CDC0D8F00001C751D96F060EDA6F97
:101F7000B1EC17F00001D890C235006E016A01364D
:101F80000A0E0024D06F000E0120D16FC251020D45
:101F9000AC0EF324E96E000EF420EA6EEF50D26F1F
:101FA000BCEC1FF00001D890C235006E016A01360A
:101FB0000B0E0024D06F000E0120D16FC251020D14
:101FC000AD0EF324E96E000EF420EA6EEF50D26FEE
:101FD000BCEC1FF00001D890C235006E016A0136DA
:101FE0000050CA0FF66E0150F76E0A0EF722040E6B
:101FF000F626000EF7220800FFFFF550890F77EC58
:1020000000F036D00501F7A301D001D031D0010E88
:102010000001C26101D001D003D0010EC22702D05D
:102020000001C26B0501F76B140E0501F86501D0C4
:1020300001D004D0080EE8CFF9F503D0140EE8CF94
:10204000F9F50001D890C235006E016A01360050E2
:10205000CA0FF66E0150F76E0A0EF722040EF6262E
:10206000000EF7220800FFFFF550890F77EC00F013
:102070000501F7A101D001D011D0010E0001C32745
:10208000080EE8CFF9F50501F76B1A0E0001D06FC5
:10209000D16BC351D26FBCEC1FF0FFD00001C65111
:1020A000D8A407D000D00501FA53D8B402D000D08C
:1020B00001D006D00501F853D8A402D000D002D038
:1020C00000D0E9D0020E98EC1AF00C0E77EC00F07C
:1020D00005014253D8B401D001D02DD00501426B87
:1020E0000001C16B010EC16501D001D001D022D029
:1020F0000001D890C135006E016A01360050CA0F48
:10210000F66E0150F76E0A0EF7220800FFFFF55039
:10211000850F77EC00F00001CE0EDC6F0B0EDD6F4B
:10212000D1EC00F0010E0001C127010EC16501D004
:1021300001D0DED794D00001C06BC16B010EC16528
:1021400001D001D001D082D00001D890C135006EFD
:10215000016A01360050CA0FF66E0150F76E0A0E82
:10216000F7220800FFFFF550850F77EC00F0000123
:10217000CA0EDC6F000EDD6FC70EDE6F000EDF6F64
:10218000C15105EE25F0E926000EEA22EF50F4ECED
:1021900016F0CAC0D7F0CBC0D8F00001C751D96F34
:1021A000060EDA6FB1EC17F00001C15105EE25F013
:1021B000E926000EEA22EF5066EC19F00001D890F3
:1021C000C135006E016A01360050CA0FF66E01502B
:1021D000F76E0A0EF722010EF626000EF72208000F
:1021E000FFFFF550800F77EC00F00001C15169EC62
:1021F00018F0040E0001C16101D001D01FD0CAC087
:10220000DCF0CBC0DDF0C751FEEC19F00001C1518C
:10221000020DB80EF324E96E000EF420EA6EEECF44
:1022200002F0EDCF03F00350015C02E10250005CCC
:10223000D8A001D001D002D0010EC06F010E000164
:10224000C127010EC16501D001D07ED70001C05168
:10225000D8B401D001D002D0898201D08992050181
:10226000FA6B0001D890C235006E016A0136005049
:10227000CA0FF66E0150F76E0A0EF722040EF6260C
:10228000000EF7220800FFFFF550890F77EC00F0F1
:102290000F0E77EC00F02EEF0DF060EF16F000015E
:1022A000C351030AD8A401D001D059D30C0E77EC46
:1022B00000F0010E77EC00F0C00E77EC00F00001AA
:1022C000120EDC6F0B0EDD6FD1EC00F0D40E77EC4C
:1022D00000F00001900EDC6F0B0EDD6FD1EC00F012
:1022E0003C0EE8CFFCF5010E0001C66FC26B89926F
:1022F00034D30001C651D8B407D000D00501FC5337
:10230000D8A402D000D002D000D0A7D0010E77EC24
:1023100000F00001C06B030EC06501D001D001D0F8
:1023200086D00001C051D06FD16BFBEC22F0006E63
:102330000001C05105EE25F0E926000EEA2200C09A
:10234000EFFFC05105EE25F0E926000EEA22EF501E
:10235000C56101D001D00ED0C05105EE25F0E926AF
:10236000000EEA22000EEF6EC051D06FD16BD26B1F
:10237000BCEC1FF0C0C000F0016A0050CA0FF66E3E
:102380000150F76E0A0EF7220800FFFFF550800F8C
:1023900077EC00F00001C05166EC16F0C0C000F010
:1023A000016A0050CA0FF66E0150F76E0A0EF7224E
:1023B0000800FFFFF550860F77EC00F00001CA0E11
:1023C000DC6F000EDD6FC70EDE6F000EDF6FC051D9
:1023D00005EE25F0E926000EEA22EF50F4EC16F0A7
:1023E0000001C051020DB80EF324E96E000EF42076
:1023F000EA6EEECFD0F0EDCFD1F0C751C6EC19F0B8
:1024000000C0CCF001C0CDF0CCC0D7F0CDC0D8F02A
:102410000001C751D96F060EDA6FB1EC17F0010E4B
:102420000001C027030EC06501D001D07AD7C2C019
:1024300000F0016A0050CA0FF66E0150F76E0A0EE6
:10244000F7220800FFFFF5508B0F77EC00F0010E2C
:10245000E8CFFAF50001C66B6AD20501F7A501D0F5
:1024600001D000D10001CA0EDC6F000EDD6FC70E77
:10247000DE6F000EDF6FC25105EE25F0E926000E7B
:10248000EA22EF50F4EC16F00001C7512DEC1AF0DF
:1024900000C0C8F001C0C9F00001C251020DB80E61
:1024A000F324E96E000EF420EA6EEECF00F0EDCFDB
:1024B00001F0C951015C02E1C851005CD8B001D003
:1024C00001D00CD0000EC95D020ED8B4C85DD8A0F2
:1024D00001D001D003D0D890C933C8330001C25114
:1024E000020DB80EF324E96E000EF420EA6EEECF72
:1024F00000F0EDCF01F00150C95D02E10050C85D70
:10250000D8B001D001D00CD0C251020DB80EF324C6
:10251000E96E000EF420EA6EC851EE5EC951ED5A24
:102520000501F76B140E0501F86501D005D0780E92
:102530000501F86102D000D002D000D004D0040E12
:10254000E8CFF9F50DD0780E0501F86501D001D07E
:1025500004D00A0EE8CFF9F503D0140EE8CFF9F550
:10256000C2C000F0016A0050CA0FF66E0150F76E4B
:102570000A0EF7220800FFFFF550860F77EC00F0F7
:102580000001CA0EDC6F000EDD6FC70EDE6F000E9D
:10259000DF6FC25105EE25F0E926000EEA22EF506A
:1025A000F4EC16F00001C251020DB80EF324E96EEE
:1025B000000EF420EA6EEECFD0F0EDCFD1F0C7518F
:1025C000C6EC19F000C0CCF001C0CDF0CCC0D7F003
:1025D000CDC0D8F00001C751D96F060EDA6FB1EC4B
:1025E00017F00001D890C235006E016A0136120E54
:1025F0000024D06F000E0120D16FC251020DB80E21
:10260000F324E96E000EF420EA6EEF50D26FBCECBA
:102610001FF00001D890C235006E016A0136130E1A
:102620000024D06F000E0120D16FC251020DB90EEF
:10263000F324E96E000EF420EA6EEF50D26FBCEC8A
:102640001FF0C2C000F0016A0050CA0FF66E0150C0
:10265000F76E0A0EF7220800FFFFF5508B0F77EC9C
:1026600000F065D10501F7A701D001D031D10001FB
:10267000CA0EDC6F000EDD6FC70EDE6F000EDF6F5F
:10268000C25105EE25F0E926000EEA22EF50ACDB40
:102690000001C7512DEC1AF000C0C8F001C0C9F00C
:1026A0000001C251020DB80EF324E96E000EF420B1
:1026B000EA6EEECF02F0EDCF03F0FF0E006EFF0EDC
:1026C000016EC851005EC951015A0350015C02E11C
:1026D0000250005CD8B001D001D00CD0000EC95D12
:1026E000020ED8B4C85DD8A001D001D003D0D890D4
:1026F000C933C833FF0E006EFF0E016E0001C851D2
:10270000005EC951015AC251020DB80EF324E96EA0
:10271000000EF420EA6EEECF02F0EDCF03F0015090
:10272000035C02E10050025CD8B001D001D00CD0B3
:10273000C251020DB80EF324E96E000EF420EA6EC9
:10274000C851EE26C951ED220501F76B140E0501A3
:10275000F86501D005D0780E0501F86102D000D0EF
:1027600002D000D004D0040EE8CFF9F50DD0780ED9
:102770000501F86501D001D004D00A0EE8CFF9F5C3
:1027800003D0140EE8CFF9F5C2C000F0016A005082
:10279000CA0FF66E0150F76E0A0EF7220800FFFF0F
:1027A000F550860F77EC00F00001C751020AD8A45B
:1027B00001D005D0C751060AD8A402D000D007D056
:1027C00000D00001C7510A0AD8A402D000D002D01C
:1027D00000D01FD00001C251020DB80EF324E96EE3
:1027E000000EF420EA6EEE52010EED5C000ED8B43D
:1027F000EF5CD8A001D001D00CD0C251020DB80EB0
:10280000F324E96E000EF420EA6EFF0EEE6E000E69
:10281000ED6E0001C251020DB80EF324E96E000EF8
:10282000F420EA6EEECFD0F0EDCFD1F0C751C6EC78
:1028300019F000C0CCF001C0CDF0CCC0D7F0CDC0B5
:10284000D8F00001C751D96F060EDA6F8ADB00019C
:10285000D890C235006E016A0136120E0024D06F86
:10286000000E0120D16FC251020DB80EF324E96EA3
:10287000000EF420EA6EEF50D26FBCEC1FF00001A6
:10288000D890C235006E016A0136130E0024D06F55
:10289000000E0120D16FC251020DB90EF324E96E72
:1028A000000EF420EA6EEF50D26FBCEC1FF0C2C0F5
:1028B00000F0016A0050CA0FF66E0150F76E0A0E62
:1028C000F7220800FFFFF5508B0F77EC00F02FD0B8
:1028D0000501F7A301D001D02AD0030E0001C26187
:1028E00001D001D003D0010EC22702D00001C26B7B
:1028F0000501F76B140E0501F86501D001D004D075
:10290000080EE8CFF9F503D0140EE8CFF9F5C2C0F0
:1029100000F0016A0050CA0FF66E0150F76E0A0E01
:10292000F7220800FFFFF5508B0F77EC00F0050150
:10293000F7A101D001D011D0010E0001C327080E6C
:10294000E8CFF9F50501F76B1A0E0001D06FD16BD6
:10295000C351D26FBCEC1FF001D0CBD4B1D1000178
:10296000C351040AD8A401D001D0AAD10C0E77EC2F
:1029700000F0010E77EC00F0C00E77EC00F00001E3
:10298000560EDC6F0B0EDD6FD1EC00F0D40E77EC41
:1029900000F00001900EDC6F0B0EDD6FD1EC00F04B
:1029A0003C0EE8CFFCF5010E0001C66FC26B8992A8
:1029B00086D10001C651D8B407D000D00501FC5320
:1029C000D8A402D000D002D000D028D0010E77ECDD
:1029D00000F00001750EDC6F0B0EDD6FD1EC00F026
:1029E000940E77EC00F00001FC0EDC6F0A0EDD6F38
:1029F000D1EC00F0D40E77EC00F00001070EDC6F94
:102A00000B0EDD6FD1EC00F00001C26B010EC46F44
:102A10000F0E77EC00F00001C66B9CD00501F7A506
:102A200001D001D036D0080EE8CFF9F50501F76BDB
:102A300025D0040E0501F66501D001D003D00501B3
:102A4000FC0EF627080E0001D06FD16BF6C5D2F050
:102A5000BCEC1FF01AD005014353D8B401D001D00B
:102A600003D00501010E435F090E0001D06FD16B49
:102A700043C5D2F0BCEC1FF008D007D00001C25112
:102A8000000AD7E0010AE7E000D0010E0001C46FA0
:102A900061D00501F7A701D001D036D0080EE8CFEC
:102AA000F9F50501F76B25D0C80E0501F66101D0D7
:102AB00001D003D00501040EF627080E0001D06FE7
:102AC000D16BF6C5D2F0BCEC1FF01AD0030E050195
:102AD000436101D001D003D00501010E4327090E47
:102AE0000001D06FD16B43C5D2F0BCEC1FF008D011
:102AF00007D00001C251000AD7E0010AE7E000D088
:102B0000010E0001C46F26D00501F7A301D001D04A
:102B100021D0010E0001C26101D001D003D0010E0D
:102B2000C22702D00001C26B080EE8CFF9F50501FB
:102B3000F76B09D0A70E77EC00F00CD0E70E77EC1E
:102B400000F008D007D00001C251000AF3E0010AEA
:102B5000F5E000D00501F7A101D001D010D00001AF
:102B6000C36B080EE8CFF9F50501F76B1A0E0001EB
:102B7000D06FD16BC351D26FBCEC1FF0A1D000015C
:102B8000C451D8B401D001D09AD09E0E77EC00F099
:102B900000012D0EEF6F050EF06F670EF16F0B0E3B
:102BA000F26FF6C5E8FF190DF3CFCEF0F4CFCFF0FA
:102BB000CE0EE8CFEDF0000EE8CFEEF001EC20F005
:102BC00000012D0EDB6F050EDC6F0A0EDD6F0EECC3
:102BD0001FF000012D0EDC6F050EDD6FD1EC00F053
:102BE000DE0E77EC00F03DD000012D0EDE6F050EFD
:102BF000DF6FE20EE06F0A0EE16FD5EC02F0370EE8
:102C00000001C56F39D000012D0EDE6F050EDF6F9C
:102C10006E0EE06F0B0EE16FD5EC02F0280E000196
:102C2000C56F2AD000012D0EDE6F050EDF6FEB0E93
:102C3000E06F0A0EE16FD5EC02F0370E0001C56FB0
:102C40001BD000012D0EDE6F050EDF6FF40EE06F5E
:102C50000A0EE16FD5EC02F0110E0001C56F0CD029
:102C60000BD043C5E8FF000ABFE0010ACCE0030A2D
:102C7000D9E0010AE6E000D000012D0EDB6F050E61
:102C8000DC6F0A0EDD6F0EEC1FF000012D0EDC6F05
:102C9000050EDD6FD1EC00F009D0A70E77EC00F047
:102CA0000CD0E70E77EC00F008D007D00001C2513D
:102CB000000AF3E0010AF5E000D00001C46B79D608
:102CC000E8EF07F00CEF00F018EF06F0FFFF8AD0F6
:102CD0000001D26F0C0E77EC00F00001D25105EE2E
:102CE00025F0E926000EEA22EF50D06F43D0000114
:102CF0002D0EDE6F050EDF6FD0510A0D4C0EF32442
:102D0000006E060EF420016E020E0024E06F000E2D
:102D10000120E16FD5EC02F038D000012D0EDE6FFE
:102D2000050EDF6FD0510A0D7C0EF324006E080EE5
:102D3000F420016E020E0024E06F000E0120E16F0E
:102D4000D5EC02F022D000012D0EDE6F050EDF6FF4
:102D5000D0510A0D160EF324006E0A0EF420016EF7
:102D6000020E0024E06F000E0120E16FD5EC02F0AE
:102D70000CD00BD043C5E8FF000AB9E0010ACDE052
:102D8000030AB5E0010ADFE000D000012D0EDF6F7D
:102D9000050EE06F8EEC1FF000500001D16F0501B1
:102DA000326B040E0001D06F0BD00001D15105EE43
:102DB0002DF0E926000EEA22200EEF6E010ED1273B
:102DC000040E0001D16501D001D0EFD700012D0E16
:102DD000DC6F050EDD6FD1EC00F00F0E77EC00F02C
:102DE0001200FFFF75D7DC00FFFFB9D00001E46FD0
:102DF0006DD00001E4510A0DF3504C0FF66EF45003
:102E0000F76E060EF722080EF626000EF7220800CF
:102E1000FFFFF550E06FE4510A0DF3504C0FF66ED2
:102E2000F450F76E060EF722010EF626000EF7227A
:102E30000800FFFFF550E16F54D00001E4510A0D86
:102E4000F3507C0FF66EF450F76E080EF722080E62
:102E5000F626000EF7220800FFFFF550E06FE45160
:102E60000A0DF3507C0FF66EF450F76E080EF72241
:102E7000010EF626000EF7220800FFFFF550E16F65
:102E800030D00001E4510A0DF350160FF66EF450E5
:102E9000F76E0A0EF722080EF626000EF72208003B
:102EA000FFFFF550E06FE4510A0DF350160FF66E78
:102EB000F450F76E0A0EF722010EF626000EF722E6
:102EC0000800FFFFF550E16F0CD00BD043C5E8FFC1
:102ED000000A8FE0010AB1E0030A8BE0010AD1E0A9
:102EE00000D012D00001E151C0EC1CF000C0E2F0B3
:102EF00001C0E3F024D00001E151F5EC1CF0000129
:102F0000E26FE36B1CD01BD00001E051000AEAE045
:102F1000010AE8E0030AEFE0010AEDE0070AE2E057
:102F2000010AE0E0030AE7E0010ADCE00F0ADAE068
:102F3000010AD8E0030ADFE0010AD4E0D3D7DCC0FD
:102F4000E9FFDDC0EAFFE2C0EEFFE3C0EDFFDEC057
:102F5000E9FFDFC0EAFFE0C0EFFF1200FFFF46D746
:102F6000D700FFFFB5D07DD000012D0EDB6F050E21
:102F7000DC6FD7C0DDF0D8C0DEF005EC1DF08ED0E0
:102F800000012D0EDB6F050EDC6FD751DD6F5CECA1
:102F90001DF084D000012D0EDB6F050EDC6FD751C4
:102FA000DD6F7AEC1DF07AD000012D0EDB6F050E7F
:102FB000DC6FD751DD6FECEC1EF070D000012D0EF0
:102FC000DB6F050EDC6FD7C0DDF0D8C0DEF09FEC04
:102FD0001DF064D000012D0EDB6F050EDC6FD7C035
:102FE000DDF0D8C0DEF070EC1EF058D000012D0EE0
:102FF000DB6F050EDC6FD7C0DDF0D8C0DEF007EC6C
:103000001EF04CD000012D0EDB6F050EDC6FD7518A
:10301000DD6FD0EC1DF042D000012D0EDB6F050EF0
:10302000DC6FD7C0DDF0D8C0DEF020EC1DF036D06C
:1030300000012D0EDB6F050EDC6FD7C0DDF0D8C0B0
:10304000DEF03BEC1DF02AD000012D0EDB6F050EEB
:10305000DC6FD7C0DDF0D8C0DEF038EC1EF01ED03B
:103060001DD00001D951000A01E17ED7010AA6E076
:10307000030A86E0010A98E0070AACE0010AB6E01C
:10308000030AC0E0010AC8E00F0AD2E0010ADCE04E
:10309000030A80E0010A01E167D766D700012D0E1F
:1030A000DB6F050EDC6FDA51DD6F0EEC1FF00001F7
:1030B000DA5105EE2DF0E926000EEA22000EEF6E41
:1030C0002D0EDC6F050EDD6FD1EC00F01200FFFF5E
:1030D0004AD7FFFF9AD00001DB6FDB5105EE25F0E8
:1030E000E926000EEA22EF50D26FD30EDC6F000EFD
:1030F000DD6FD00EDE6F000EDF6FD25175DED3C0F4
:10310000DCF0D4C0DDF00001D05178D900C0D5F09A
:1031100001C0D6F0280E046E056A066A076AD5C09B
:1031200000F0D6C001F0026A036A51EC02F000011F
:10313000DB51020DAC0EF324E96E000EF420EA6EB2
:10314000EECFF6FFEDCFF7FFF650046EF750056EA9
:10315000066A076AF3EC01F000C0D7F001C0D8F0AE
:1031600002C0D9F003C0DAF0D751D16FD06B130E83
:10317000D06501D001D001D010D00001D05105EEB2
:103180002DF0E926000EEA22200EEF6E010ED02768
:10319000130ED06501D001D0F0D70001D06B270EFF
:1031A000D06501D001D001D025D00001D151D0632C
:1031B00001D001D00ED0D1A101D001D009D0D8903A
:1031C000D03105EE2DF0E926000EEA22020EEF6E58
:1031D00011D00001D890D03105EE2DF0E926000E77
:1031E000EA22010EEF6E010ED027270ED06501D026
:1031F00001D0DBD70501416B00012D0EDC6F050E00
:10320000DD6FD1EC00F01200FFFF65D7FFFF5DD04E
:103210000001D66FD65105EE25F0E926000EEA2210
:10322000EF50D16FD20EDC6F000EDD6FD00EDE6F6F
:10323000000EDF6FD151D8DDD2C0DCF0D3C0DDF09D
:103240000001D051DBD800C0D4F001C0D5F000019E
:10325000D651020DB00EF324E96E000EF420EA6E92
:10326000EECF00F0EDCF01F00150D55D02E100504E
:10327000D45DD8A001D001D00DD0D651020DB00E32
:10328000F324E96E000EF420EA6ED4C0EEFFD5C040
:10329000EDFF01D018D0040EA1EC00F00001D20E19
:1032A000DC6F000EDD6FD00EDE6F000EDF6FD151D0
:1032B0009BDDD2C0D7F0D3C0D8F00001D051D96F78
:1032C000050EDA6F4EDE1200FFFFA2D7FFFF5CD0C3
:1032D0000001D16F3AD00001D1510A0DF3504C0FCB
:1032E000F66EF450F76E060EF722090EF626000E63
:1032F000F7220800FFFFF550D06F32D00001D15106
:103300000A0DF3507C0FF66EF450F76E080EF7229C
:10331000090EF626000EF7220800FFFFF550D06FC9
:103320001FD00001D1510A0DF350160FF66EF45064
:10333000F76E0A0EF722090EF626000EF722080095
:10334000FFFFF550D06F0CD00BD043C5E8FF000A4B
:10335000C2E0010AD3E0030ABEE0010AE2E000D0C5
:10336000D0C000F0016AD89000360136D8900036FF
:103370000136000E00240001DC6F060E0120DD6F17
:10338000D1EC00F01200FFFFA3D7D000FFFF34D034
:103390000001D56F23D00001000ED025D26F800E22
:1033A000D121D36F22D00001810ED025006EFF0EF7
:1033B000D121016E001E011E002AD8B4012A00C0CE
:1033C000D2F001C0D3F0D251D46FD451D26FD36BAD
:1033D0000CD0D0C0D2F0D1C0D3F007D00001D5516D
:1033E000000AD9E00A0ADFE0F4D7D2C000F0D3C067
:1033F00001F000D01200FFFFCBD7DC00FFFF2CD084
:103400000001E16F1BD00001000EDC25DE6F800E95
:10341000DD21DF6F1AD00001DC51E06FE0510008C0
:10342000DE6FDF6BDEBFDF077F0EDE27000EDF23E0
:103430000CD0DCC0DEF0DDC0DFF007D00001E151D0
:10344000000AE1E00A0AE7E0F4D7DEC000F0DFC0DE
:1034500001F000D01200FFFFD3D7FFFF68D00001BA
:10346000D26F4DD0010E0001D06FD16B770E0501E8
:10347000F86501D001D004D0140E0001D06FD16BDB
:103480004FD0010E0001D06FD16B770E0501F865AA
:1034900001D001D004D00A0E0001D06FD16B40D012
:1034A0000A0E0001D06FD16B770E0501F86501D0CF
:1034B00001D004D0640E0001D06FD16B31D0080E62
:1034C0000001D06FD16B770E0501F86501D001D0F6
:1034D00004D0500E0001D06FD16B22D0010E00013C
:1034E000D06FD16B770E0501F86501D001D005D002
:1034F0000001000ED06F010ED16F12D011D000016B
:10350000D251020AAFE0060ADAE0010ABAE0030A81
:10351000A9E00F0AC5E0030AA5E0010AA3E0DED78F
:10352000D0C000F0D1C001F000D01200FFFF97D74B
:10353000FFFFAFD00001D26BD06BD36F6DD04FD0F7
:103540000001D05105EE25F0E926000EEA22EF50E9
:103550000A0DF3504C0FF66EF450F76E060EF7227C
:10356000010EF626000EF7220800FFFFF550F00BC3
:10357000D16F40D00001D05105EE25F0E926000EB4
:10358000EA22EF500A0DF3507C0FF66EF450F76EFE
:10359000080EF722010EF626000EF7220800FFFFA4
:1035A000F550F00BD16F26D00001D05105EE25F07B
:1035B000E926000EEA22EF500A0DF350160FF66EC0
:1035C000F450F76E0A0EF722010EF626000EF722CF
:1035D0000800FFFFF550F00BD16F0CD00BD043C5A6
:1035E000E8FF000AADE0010AC5E0030AA9E0010A0C
:1035F000DBE000D00001D13B0F0ED117D1C001F0AC
:10360000010E006E012A02D0D8900036012EFCD7A0
:103610000050D213010ED0270001D351D05DD8A0A5
:1036200001D001D08CD70001D06B070ED06501D03E
:1036300001D001D028D0D0C001F0010E006E012AC7
:1036400002D0D8900036012EFCD70001D2510014D0
:103650000009D8B401D001D00ED0D039F00BD16F11
:10366000D15156EC1CF005014253D8B401D001D021
:1036700002D089900CD0010E0001D027070ED06532
:1036800001D001D0D8D78980280EE8CFF4F51200F8
:10369000FFFF50D7FFFF0CD0330EAF6E240EAC6E81
:1036A000900EAB6E949C948E0501426B1200FFFF4E
:1036B000F3D7FFFF0DD00001DE6F01D000D09EA830
:1036C00001D001D0FBD70001DE51AD6E1200FFFF2B
:1036D000F2D7FFFF16D0040EE8CFF5F50AD00501AA
:1036E000F553D8A401D001D004D0010EE8CF42F5A3
:1036F00004D09EAA01D001D0F2D7AE5000D0120063
:10370000FFFFE9D7FFFF23D00001DE6B170EDE6558
:1037100001D001D001D019D0100EE8CFF5F507D0B7
:103720000501F553D8A401D001D001D00ED09EAA36
:1037300001D001D0F5D7AE500001DF6F010EDE27BA
:10374000170EDE6501D001D0E7D71200FFFFDCD7EE
:10375000D900FFFFAAD031D03C0EE8CF5CF50501BF
:103760005F6BDBC060F5DAC061F5D9C062F530D0BF
:10377000A50EE8CF5CF50501606BDBC05FF5D9C035
:1037800061F5DAC062F524D0A50EE8CF5CF505013D
:103790005F6BDBC060F5DAC061F5D9C062F518D0A7
:1037A0005A0EE8CF5CF50501606BDBC05FF5D9C050
:1037B00061F5DAC062F50CD00BD043C5E8FF000A12
:1037C000CBE0010AD5E0030ADFE0010AE9E000D01E
:1037D0003A0EE8CF5DF5100EE8CF5EF5070E00015A
:1037E000DC6F170EDC6501D001D001D010D00001D4
:1037F000DC5105EE5CF0E926000EEA22000EEF6EC9
:10380000010EDC27170EDC6501D001D0F0D70001D6
:10381000DD6B5CC5E8FF4DDF010E0001DC6F160EAD
:10382000DC6501D001D001D019D00001DC5105EEDA
:103830005CF0E926000EEA22EF503BDF0001DC518C
:1038400005EE5CF0E926000EEA22EF50DD27010EBE
:10385000DC27160EDC6501D001D0E7D70001DD5171
:10386000000827DF0001DC6B170EDC6501D001D0FA
:1038700001D019D00001DC5105EE44F0E926000E1C
:10388000EA2227DFEF6E05014253D8B401D001D000
:1038900002D038DF08D0010E0001DC27170EDC65EE
:1038A00001D001D0E7D71200FFFF55D7FFFF67D047
:1038B0000001D86FD851F00BD76F27D00001000E50
:1038C000D725D46FD56B400ED523800ED66F28D068
:1038D0000001000ED725D46FD56BEF0ED523D66926
:1038E0001FD00001000ED725D46FD56B400ED52315
:1038F000800ED66F15D00001000ED725D46FD56B82
:10390000FC0ED523D66B0CD00BD043C5E8FF000AC4
:10391000D5E0010ADDE0030AE4E0010AECE000D0B2
:10392000D4C0D9F0D5C0DAF00001D651DB6F11DF79
:103930000001D66B0F0ED66501D001D001D01DD08D
:103940000001D65105EE4BF0E926000EEA22D651D1
:10395000D7C000F0016A0026000E0122740E002478
:10396000E16E050E0120E26EEFCFE7FF010ED627D4
:103970000F0ED66501D001D0E3D71200FFFF98D714
:10398000FFFF32D00001E76F43C5E8FF030AD8A468
:1039900001D001D011D0E75105EE74F0E926000EF8
:1039A000EA22EF50E56FE75105EE75F0E926000ECB
:1039B000EA22EF50E66F11D00001E75105EE75F0F5
:1039C000E926000EEA22EF50E56FE75105EE74F0AC
:1039D000E926000EEA22EF50E66FE5C000F0E6C0EF
:1039E00001F000D01200FFFFCDD7FFFF0CD0000187
:1039F000E56FE55105EE74F0E926000EEA22EF507E
:103A000000D01200FFFFF3D7DB00FFFF17D0DBC0B1
:103A1000EFF0DCC0F0F00001FF0EF16F0B0EF26F63
:103A2000DDC0DFF0DEC0E0F0DF0EE8CFEDF0000E2D
:103A3000E8CFEEF001EC20F01200FFFFE8D7DB004A
:103A4000FFFF17D0DBC0EFF0DCC0F0F00001FB0E91
:103A5000F16F0B0EF26FDDC0DFF0DEC0E0F0DF0EC5
:103A6000E8CFEDF0000EE8CFEEF001EC20F0120010
:103A7000FFFFE8D7DB00FFFF1DD0DBC0EFF0DCC0AD
:103A8000F0F00001FF0EF16F0B0EF26FCE0EDD2590
:103A9000006EFF0EDE21016E00C0DFF001C0E0F01D
:103AA000DF0EE8CFEDF0000EE8CFEEF001EC20F0F5
:103AB0001200FFFFE2D7DB00FFFF1AD0DBC0EFF000
:103AC000DCC0F0F00001030EF16F0C0EF26FDDC0F0
:103AD00000F0016A00C0DEF001C0DFF0DE0EE8CFCA
:103AE000EDF0000EE8CFEEF001EC20F01200FFFF49
:103AF000E5D7DB00FFFF21D0DBC0EFF0DCC0F0F04A
:103B00000001030EF16F0C0EF26FDDC000F0016AD0
:103B100000BE0106001E011E002AD8B4012A00C002
:103B2000DEF001C0DFF0DE0EE8CFEDF0000EE8CFF2
:103B3000EEF001EC20F01200FFFFDED7DB00FFFF0C
:103B40002DD0DBC0EFF0DCC0F0F000011A0EF16FF9
:103B50000C0EF26F0A0E026E036ADDC000F0DEC0CA
:103B600001F058EC1FF000C0E1F001C0E2F00A0ED5
:103B7000026E036ADDC000F0DEC001F058EC1FF0F9
:103B800004C0DFF005C0E0F0DF0EE8CFEDF0000E7E
:103B9000E8CFEEF001EC20F01200FFFFD2D7DB00FF
:103BA000FFFF33D00001DD51050DF3CFDEF0F4CF80
:103BB000DFF0DBC0EFF0DCC0F0F01A0EF16F0C0E9E
:103BC000F26F0A0E026E036ADEC000F0DFC001F081
:103BD00058EC1FF000C0E2F001C0E3F00A0E026EE4
:103BE000036ADEC000F0DFC001F058EC1FF004C033
:103BF000E0F005C0E1F0E00EE8CFEDF0000EE8CF18
:103C0000EEF001EC20F01200FFFFCCD7DB00FFFF4D
:103C10002DD0DBC0EFF0DCC0F0F00001070EF16F3B
:103C20000C0EF26F640E026E036ADDC000F0DEC09F
:103C300001F058EC1FF000C0E1F001C0E2F0640EAA
:103C4000026E036ADDC000F0DEC001F058EC1FF028
:103C500004C0DFF005C0E0F0DF0EE8CFEDF0000EAD
:103C6000E8CFEEF001EC20F01200FFFFD2D7DB002E
:103C7000FFFF34D0DBC0EFF0DCC0F0F00001070E36
:103C8000F16F0C0EF26FE80E026E030E036EDDC0D4
:103C900000F0DEC001F058EC1FF00A0E026E036A5D
:103CA00058EC1FF004C0E1F005C0E2F0E80E026E2F
:103CB000030E036EDDC000F0DEC001F058EC1FF013
:103CC00004C0DFF005C0E0F0DF0EE8CFEDF0000E3D
:103CD000E8CFEEF001EC20F01200FFFFCBD7DB00C5
:103CE000FFFF78D0670E046E350E056E000E066E6F
:103CF000000E076EDDC000F0DEC001F0026A036A4C
:103D000051EC02F000C0DFF001C0E0F002C0E1F0D1
:103D100003C0E2F0A00E046E860E056E010E066E64
:103D2000000E076EDFC000F0E0C001F0E1C002F05D
:103D3000E2C003F0DFEC1FF09C0E00240001E36FF3
:103D4000FF0E0120E46FE3C0EDF0E4C0EEF03EECC6
:103D500023F000C0E5F001C0E6F0DBC0EFF0DCC00E
:103D6000F0F00001100EF16F0C0EF26F640E026E97
:103D7000036AE5C000F0E6C001F015EC23F000C0D6
:103D8000EBF001C0ECF0640E026E036AE5C000F0D7
:103D9000E6C001F015EC23F004C0E9F005C0EAF03C
:103DA000E4BF09D000D0200E006E016A05D02D0EB0
:103DB000006E016A01D0FBD700C0E7F001C0E8F057
:103DC000E70EE8CFEDF0000EE8CFEEF001EC20F0CA
:103DD0001200FFFF87D7DB00FFFF1ED00001DD517F
:103DE000D8B401D001D00BD0DBC0DEF0DCC0DFF0F6
:103DF000220EE06F0C0EE16FD5EC02F00BD0DBC0B1
:103E0000DEF0DCC0DFF00001250EE06F0C0EE16F8C
:103E1000D5EC02F01200FFFFE1D7DB00FFFF47D037
:103E2000DBC0DFF0DCC0E0F08EEC1FF000500001E2
:103E3000DE6FDD51DE5DD8A001D001D001D035D0DC
:103E40000001DD51DB25E96E000EDC21EA6E000E7B
:103E5000EF6E13D0010E0001DD5F010EDE5FDE515B
:103E6000DB25E16E000EDC21E26EDD51DB25E96E23
:103E7000000EDC21EA6EE7CFEFFF0001DE51D8A48F
:103E800001D001D0E7D70BD0010E0001DD5FDD517D
:103E9000DB25E96E000EDC21EA6E200EEF6E0001DC
:103EA000DD51D8A401D001D0EFD71200FFFFB8D761
:103EB000FFFF066AFFFF046A056A0250031003E170
:103EC000006A016A000C1F0E0612D890062A0236FC
:103ED0000336FCE3033202320250005C0350015807
:103EE00004E3016E0250005ED88004360536062ECB
:103EF00006BAF0D706AE05D0041E042AD8B40506CB
:103F0000051E0450026E0550036E06AC000C001E28
:103F1000002AD8B40106011E000CDF00FFFFDFC03D
:103F2000F3FFE0C0F4FFF3CFF6FFF4CFF7FFF32A7F
:103F3000000EF422050EF76404D00800FFFFF550D0
:103F400005D0F6CFE9FFF7CFEAFFEF500009D8A47C
:103F5000EAD7F3CF00F0F4CF01F00001DF51005EAB
:103F6000E051015AFF0E0024006EFF0E0120016E89
:103F70001200FFFFD4D7D000FFFFA6B2FED700018A
:103F8000D051A96ED251A86E3F0EA616D890F2BE9F
:103F9000D880F29ED892F2BCD882F29CA684550EAC
:103FA000A76EAA0EA76EA682A6B2FED7A198A69467
:103FB000D8B0F28ED8B2F28C1200FFFFDED7FFFF2E
:103FC000E96AEA6AFFFF0C6A03AE04D05DEC23F0F5
:103FD0000C8C0C8E0750800B0C1A07AEF8EF01F01A
:103FE000D890FF0E0406041ED8A00526051ED8A0F2
:103FF0000626061ED8A00726071EF8EF01F0FFFFD1
:10400000ED00FFFF0001FB6BFC6BEDC0F9F0EEC0B3
:10401000FAF00001F1C0F6FFF2C0F7FFF12B000E3D
:10402000F223050EF76404D00800FFFFF55005D019
:10403000F6CFE9FFF7CFEAFFEF50F66FF651000138
:10404000D8B4C7D2250AD8B40BD0FB2B000EFC2362
:10405000F051EF11D8A47BD1F65171EC23F0D9D7F0
:104060000001F469F56BF36B62D20001F051EF11BE
:10407000D8A4B3D2B8D2F9C0E9FFFAC0EAFF000170
:10408000020EF927000EFA23EF5095D20001F38DAE
:104090004ED20001F32B06D0080E0001F427FE0ECD
:1040A0000001F427F9C0E9FFFAC0EAFF0001020E9F
:1040B000F927000EFA23EECFF7F0EDCFF8F0F3A1D9
:1040C0000DD0F8AF06D0F76DF81FD8B0F82BF50774
:1040D00007D00001F391F3AD03D0F9D70001F391BC
:1040E0000B0E0001F427F4C002F0036AF7C000F0E1
:1040F000F8C001F058EC1FF000500001F66FF4C05A
:1041000002F0036AF7C000F0F8C001F058EC1FF0AD
:1041100004C0F7F005C0F8F0010EFD6FFE6B000162
:10412000FE51F85D02E1FD51F75DD8A010D0F4C05A
:1041300002F0036AFDC000F0FEC001F04EEC23F077
:1041400004C0FDF005C0FEF00001F507E8D700014E
:10415000F3A916D01CD00001FB2B000EFC23F0515C
:10416000EF11D8B40AD0EFC0E9FFF0C0EAFF200E8B
:10417000EF6EEF2B000EF02303D0200E71EC23F036
:104180000001F507F551800A7F0FD8B0E4D7000190
:10419000F3A115D0FB2B000EFC23F051EF11D8B486
:1041A0000AD0EFC0E9FFF0C0EAFF2D0EEF6EEF2B53
:1041B000000EF02317D02D0E71EC23F013D0000168
:1041C000F3AD10D0FB2B000EFC23F051EF11D8B44F
:1041D00006D0EFC0E9FFF0C0EAFF2B0EE7D72B0EA9
:1041E00071EC23F00001F3B916D051D00001FB2B84
:1041F000000EFC23F051EF11D8B40AD0EFC0E9FF54
:10420000F0C0EAFF300EEF6EEF2B000EF02303D06C
:10421000300E71EC23F00001F507F551800A7F0F95
:10422000D8A035D0E3D7FDC002F0FEC003F0F7C040
:1042300000F0F8C001F058EC1FF004C000F005C019
:1042400001F0F4C002F0036A58EC1FF000500001C6
:10425000F56F800A760FD8A002D0070EF52700016F
:10426000FB2B000EFC23F051EF11D8B40BD0F5510D
:10427000300FEFC0E9FFF0C0EAFFEF6EEF2B000E4A
:10428000F02305D00001F551300F71EC23F0F4C09C
:1042900002F0036AFD0EE96E000EEA6EEE50006E4B
:1042A000EF50016E58EC1FF00550ED6E0450EF6EAC
:1042B000EE50ED10D8A4B7D7090E0001F66502D074
:1042C000070EF6270001FB2B000EFC23F051EF1127
:1042D000D8B408D0F651300FEFC0E9FFF0C0EAFFC4
:1042E000EF6E3BD00001F651300F71EC23F091D608
:1042F0000001F551800A7E0FD8A017D0FB2B000ECD
:10430000FC23F051EF11D8B40AD0EFC0E9FFF0C0A0
:10431000EAFF200EEF6EEF2B000EF02303D0200EED
:1043200071EC23F00001F507E3D7F9C0E9FFFAC00B
:10433000EAFF0001020EF927000EFA23EF50F66F94
:10434000FB2B000EFC23F051EF11D8B40AD0EFC0C4
:10435000E9FFF0C0EAFFF6C0EFFFEF2B000EF023FD
:1043600058D60001F65171EC23F053D6F9C0E9FF9D
:10437000FAC0EAFF0001020EF927000EFA23EECF81
:1043800000F0EDCF01F000C0AAF001C0ABF0D96A97
:10439000AAC000F0ABC001F0D9500024026E000E9C
:1043A0000120036E02C0F6FF03C0F7FF050EF7649D
:1043B00004D00800FFFFF55005D0F6CFE9FFF7CF96
:1043C000EAFFEF500009D8B402D0D92AE1D70001A2
:1043D000F451D96002D0D950F46F0001F451F5BF07
:1043E00046D0FF0AF525D8A042D0FB2B000EFC23B7
:1043F000F051EF11D8B40AD0EFC0E9FFF0C0EAFFE6
:10440000200EEF6EEF2B000EF02303D0200E71EC88
:1044100023F00001F507E1D7AAC0F6FFABC0F7FF14
:10442000050EF76404D00800FFFFF55005D0F6CF65
:10443000E9FFF7CFEAFFEF500001F66F0001AA2B6A
:10444000000EAB230001FB2BFC23F051EF11D8B47D
:104450000AD0EFC0E9FFF0C0EAFFF6C0EFFFEF2B94
:10446000000EF02304D00001F65171EC23F000019E
:10447000F407F429D8B4CDD5CFD7F1C0F6FFF2C0F8
:10448000F7FF050EF76404D00800FFFFF55005D0D4
:10449000F6CFE9FFF7CFEAFFEF502A0AD8A40FD0F2
:1044A000F9C0E9FFFAC0EAFF0001020EF927000E89
:1044B000FA23EF50F46FF12B000EF22338D0F1C045
:1044C000F6FFF2C0F7FF050EF76404D00800FFFF07
:1044D000F55005D0F6CFE9FFF7CFEAFFEF50D00F48
:1044E0000001F46FF12B000EF223F1C0F6FFF2C0D1
:1044F000F7FF050EF76404D00800FFFFF55005D064
:10450000F6CFE9FFF7CFEAFFEF50D96E2F0ED9644F
:104510000ED03A0ED9600BD00001F4510A0DD950DB
:10452000F324D00FC7D70001F3B538D0F3890001C9
:10453000F1C0F6FFF2C0F7FFF12B000EF223050EDB
:10454000F76404D00800FFFFF55005D0F6CFE9FF6F
:10455000F7CFEAFFEF50F66F000A01E186D52A0A8D
:1045600001E189D5010A01E191D5050A86E01E0A1B
:10457000DAE0680A01E190D53B0A01E1B9D6070A01
:1045800001E187D50B0A01E18AD51C0A01E1EED6CB
:10459000060A01E187D50D0A01E17ED52F0E000143
:1045A000F6650BD03A0EF66108D0F385F5510A0D89
:1045B000F651F324D00FF56FBAD70001FB2B000E94
:1045C000FC23F051EF11D8A4C2D6F65171EC23F0C0
:1045D00020D5F051EF11D8B406D0EFC0E9FFF0C0FC
:1045E000EAFF000EEF6AFBC000F0FCC001F0120011
:1045F000FFFF08D5D000FFFF0001D051A96ED89071
:10460000F2BED880F29ED892F2BCD882F29C3F0EC5
:10461000A616A680A850D06FD16BD8B0F28ED8B2B3
:10462000F28CD0511200FFFFE7D7FFFF066A01AE00
:1046300006D0001E004A0106011E068C068E03509D
:10464000800B061A03AE5AEF1FF0021E024A030641
:10465000031E5AEF1FF0FFFF036A026A016A006A35
:10466000FFFFE950EA1008E003C0EDFF02C0EDFFD4
:1046700001C0EDFF00C0EFFF000CED00FFFF0001E7
:10468000EDC000F0EEC001F0EEAF05D0001E011E3F
:10469000002AD8B4012A1200FFFFF1D7FFFF025011
:1046A0000002F3CF04F0F4CF05F00102F350052629
:1046B00003500002F35005261200FFFF001E011EEA
:1046C000021E031E000E002A0122022203221200F3
:1046D000EE6AFFFFEA50E262FBD7E950E162F8D7E9
:1046E0001200FFFF1200FFFFFDD7FFFFFFFFFFFFDC
:1046F000FFFFFFFFFFFFFFFFFFFFFFFFFFFFFFFFCA
:00000001FF
